:03000000021104E6
:03000B000200A54B
:03002B000202AE20
:03005B0002045F3D
:030073000204394B
:1000800002030406080C10182030406080040608A3
:100090000C10182030406080A0C00D0D0403060D28
:1000A0000503030202C2AFC0D0C0E020620C20688A
:1000B00002419D306602415DE47385258AC262E596
:1000C00025F4700221242068022111207210758B02
:1000D00000D0E0D0D0C2B1C287C281D2AF32C2B1AB
:1000E000C287C2817406D5E0FDE53C1420E21520EC
:1000F000E10D207D02D280307D02D282020121D228
:1001000086020121207D02D282307D02D28002014E
:1001100021758B00D0E0D0D0C2B1C287C281D2AFEE
:1001200032758B00D0E0D0D0D2AF32419DE5256052
:100130000A207D02D2B1307D02D281C287419DE585
:10014000256002D287207D02C281307D02C2B1418A
:100150009DE525600A207D02D281307D02D2B1204A
:100160007D02C2B1307D02C281419D207D02C282EA
:10017000307D02C280207D02C280307D02C2827446
:1001800006D5E0FDE525600A207D02D2B1307D0272
:10019000D281C287419D207D02C282307D02C28011
:1001A000C2867406D5E0FDE525600A207D02D2B145
:1001B000307D02D281C287419DC286207D02C282EB
:1001C000307D02C2807406D5E0FDE5256002D2874D
:1001D000207D02C281307D02C2B1419DC286207D58
:1001E00002C280307D02C2827406D5E0FDE5256042
:1001F00002D287207D02C281307D02C2B1419D20A2
:100200007D02C280307D02C282C2867406D5E0FDC6
:10021000E525600A207D02D281307D02D2B1207DA9
:1002200002C2B1307D02C281419D207D02C2803078
:100230007D02C282207D02C282307D02C2807406AD
:10024000D5E0FDE525600A207D02D281307D02D215
:10025000B1207D02C2B1307D02C281419D30723D2C
:10026000E53C20E21A20E129207D02C282307D0295
:10027000C280207D02C280307D02C28202029D20A7
:10028000E1E6207D02C282307D02C280C286020287
:100290009DC286207D02C280307D02C282E525F4A7
:1002A000F58A758B00D262D0E0D0D0D2AF32C2AF27
:1002B000C2AD53E6EFC0D0C0E0D2D3D2AFC2CEE5DC
:1002C0002960072074461529610C78007900E580C3
:1002D000307E01F430E50278FF53DACF207E03430D
:1002E000DA20307E0343DA10C2D8C271E580307E56
:1002F00001F430E50279FFC3E89970CE30610375EF
:1003000029402074037529408859D270E52A600479
:10031000152A611C20740543DA01C2D820700261DD
:1003200044A859206102C270207402612D882230D5
:10033000690AC3E522955E4003855E227882B60491
:1003400003852224C3E52594404002D26420CF0CCB
:10035000D0E0D0D0C2D343E610D2AD32C2CF7802C3
:10036000E52960053074021529C3E559940140055B
:10037000755C006186755D00756400E55C2401F5BF
:100380005C5003755CFF7982B7020EE547601EC3BF
:10039000E522943240178546227982B7030FE5475C
:1003A000600BC3E52294324004798E8722C3E52393
:1003B000952260084004152361BC0523D8C8056454
:1003C000E56470021564D565647565017805C3E55B
:1003D0006495664058C3E564956750087801756573
:1003E000030203F0C3E56495685005780175650163
:1003F000C3E55F9524401F7982B704028122E54757
:10040000701485245FE56404600385666475650186
:1004100075233C02042DE55F285005755FFF81229E
:10042000F55FE55F047006755DFF7564FFD0E0D091
:10043000D0C2D343E610D2AD32C0D0C0E0C2AF5379
:10044000917F53E67FC260759100C3E49550F594A7
:10045000E49551F595759104D0E0D0D0D2AF32C279
:10046000AF53E6EFC2ADC0D0C0E0C0F0D2D3D2AF40
:0E047000A8FBA9FCC2D830710281C653DACFB6
:10047E00207E0343DA10307E0343DA20D271E5800A
:10048E00307E01F420E502819D88268927C19D5387
:10049E00DACF207E0343DA20307E0343DA10C2D84F
:1004AE00C271307402C1897800E580307E01F4306B
:1004BE00E502C1898859C17053DACF207E0343DA31
:1004CE0020307E0343DA10C271206102A19653DA06
:1004DE00CF207E0343DA10307E0343DA20C2D8D217
:1004EE007188548955C3E89552F8E99553F9E4FBA0
:1004FE007E027A00C3E8948CE9940050057558008A
:10050E00A186C3E894C8E994005008E4D2E4FB7ACB
:10051E000AA163C3E89468E994015008E4D2E3FBAE
:10052E007A0FA163C3E894D0E994025008E4D2E2B2
:10053E00FB7A1EA163C3E894A0E994055008E4D2A7
:10054E00E1FB7A3CA163C3E89498E994085008E46F
:10055E00D2E0FB7A787E00C3E89556FCE99557FD0C
:10056E0030E708ECF42401FCEDF4FD755800C3EC03
:10057E009AED9E500375580188568957A854A9556F
:10058E00885289537802C170C3E89526F8E99527F9
:10059E00F9307C02C154307B02C154307A02C14D15
:1005AE00207502A1B9E9FDE8FCA1D8E9C313F9E869
:1005BE0013F8307902C14DE9C313F9E813F8307816
:1005CE0002C14DE9C313FDE813FC206126C3EC9470
:1005DE001CED94024002A1EFED7018C3EC94C850CC
:1005EE00120528C3E528940A5002C189755900D214
:1005FE0070C189E528600215287400207F03789663
:10060E00E624FAFEE43400FFC3EC9EFCED9FFD50A1
:10061E000678007900C154C3EC94FFED94004006B7
:10062E0078FF7900C154EC856FF0A4C5F0A2F733C2
:10063E00F87900400302067078FF7900020670E92F
:10064E00C313F9E813F8307C0EE9600278FFC3E8B3
:10065E001338F8E43400F9C3E894FFE9940040023B
:10066E0078FF8859D270206102C189741FF4552F0A
:10067E004BF52FC274E42B7002D27475294030747E
:10068E000375290A306102C19D20740353DAFE7589
:10069E002A20307403752A0AD0F0D0E0D0D0C2D30D
:1006AE00D2AD43E6103279010206D279030206D2A8
:1006BE00790A0206D2791E0206D279640206D2792E
:1006CE00C80206D27817E4D5E0FDD8FAD9F6227A18
:1006DE00147B780206F97A107B8C0206F97A0D7B70
:1006EE00B40206F97A0B7BC80206F9AC2575250112
:1006FE007902B27DE4C286D5E0FDE5256002D2879F
:10070E00D5E0FDC287D5E0FDD286D5E0FDE52560BA
:10071E000A207D02D2B1307D02D281E570D5E0FD96
:10072E00207D02C2B1307D02C2817496D5E0FDD922
:10073E00C1EAF8D5E0FDD8FBDBB1C2868C2522C319
:10074E007C007D0075F00005F0EA33FAEB33FB50C8
:10075E00F6EB13FBEA13FAC3E9FFE8FEE89AF8E9B1
:10076E009BF95004EFF9EEF8B3EC33FCED33FDD505
:10077E00F0DFEDF9ECF822E889F08A20D2D4F8A95E
:10078E00F07B0030F70B7BFFF42401F8E9F4340022
:10079E00F9E88520F0A4ADF0F8E98520F0A4AFF0DB
:1007AE00FEED2EF974003FFA7C04C3EA13FAE91346
:1007BE00F9E813F8DCF48BF030F70AE8F42401F8CA
:1007CE00E9F43400F9E889F0C2D4F8A9F02278826D
:1007DE00B6040302087EC3E5599419401FE52D5453
:1007EE00067019E547703878057994E71460077834
:1007FE000A1460027812C3E53B984020E547600971
:10080E0085615F7564FF756501852224E4F53EF50B
:10081E003FF540F541F542F54702087E75470179EF
:10082E0094E7147013E523F43333F913F8E9540104
:10083E0004F9E854FE020872E714147014E523F468
:10084E00333333F913F8E9540304F9E854FC02087E
:10085E007AE523F433333333F913F8E954070404F8
:0E086E00F9E854F8C39440F8E99400F9883E84
:10087C00893F22E547603BC3E53B13F9E53A13F8A2
:10088C00C3E53E98F8E53F99F9500CC3E89480E92C
:10089C0094FF40160208BAC3E8947FE99400500311
:1008AC000208BA787F79000208BA788079FF884309
:1008BC00894422E5476058E5432540F8E544354135
:1008CC00F9854420E4300701F43542FA30E709C3D6
:1008DC00EA94F040150208FCC3EA940F5003020896
:1008EC00FC78FF79FF7A0F0208FC780079007AF027
:1008FC00C3E524955E5006E52460092115E54420E6
:10090C00E70D2115E54430E706884089418A4222EB
:10091C00E547700302098078A1E6FAC3E54333F892
:10092C00E54433F9120785E930E70BC3E89480E915
:10093C0094FF40132157C3E8947FE994005002219F
:10094C0057787F79002157788079FFE820E715C325
:10095C00E52398F84009C3E89401400302097E7826
:10096C000102097EE8F424012523F8400302097EE4
:10097C0078FF884522E54770030209E378A2E6FA7E
:10098C00A841A942120785E930E70CC3E89401E9B4
:10099C0094FF40160209BAC3E894FFE9940050038F
:1009AC000209BA78FF79000209BA780179FFE920C7
:1009BC00E715C3E54598F84009C3E89401400302E4
:1009CC0009E178000209E1E8F424012545F8400327
:1009DC000209E178FF88242278FFC264E52D5406D1
:1009EC00702FD264C3E53B940A4009C3E5259440BB
:1009FC005002C264E53B601974FF853BF084853777
:100A0C00F0A4F8C5F0600278FFC3E895615002A825
:100A1C00618860227883E6F520120F2075E8901229
:100A2C0006B475E890E5E820ECFBA8BDA9BE120F52
:100A3C00A0756B55756C00C3740013FD745513FCD5
:100A4C0074552CFC74003DFDECFAEDFBC3E89AE9FF
:100A5C009B4014E56B2455F56BE56C3400F56CEAA2
:100A6C002CFAEB3DFB80E5AE6BAF6CC3E56C13F978
:100A7C00E56B13F8C3E913F9E813F8E56B28F5698E
:100A8C00E56C39F56A7A03C3E913F9E813F8DAF778
:100A9C00AA201A7009756B00756C00020ABA1AEA62
:100AAC006008EE28FEEF39FFDAF88E6B8F6C22753A
:100ABC00E890227883E6FFE5E820ECF7A8BDA9BE14
:100ACC00056DC3E56D94084052756D00E9FA79A087
:100ADC00E76044EA7007E56E601B020AF5C3E8950F
:100AEC006E6010E56E5006600C14020B010460F988
:100AFC00020B01E56EF56EC394A8401B755EC0C376
:100B0C0094054013755E80C39405400B755E40C31D
:100B1C0094054003755E0075BB0622EFC39401601B
:100B2C001BC3E894FFE994035012C3E8956BE99555
:100B3C006C5009E55E600C155E020B4FE55EF460CF
:100B4C0002055EA85EC3E524985002A824C3E8956C
:100B5C005F400AA85FE55FF46003855F5E8825E56A
:100B6C006DB4070375BB1E22743279A387F0A4C53C
:100B7C00F0A2F733F8C3E8955E4002A85E8822889D
:100B8C00248825886122753A00753B7F2275C82020
:100B9C00A8CCA9CD75C824AA38AB3988388939C3F3
:100BAC00E89AF8E99BF9AA3AAB3BAC3AAD3B7E0428
:100BBC007F02C3EB940440021E1FC3EB9408400257
:100BCC001E1FC3ED13FDEC13FCDEF7C3EA9CFAEB1E
:100BDC009DFBEF6009C3E913F9E813F8DFF7EA2886
:100BEC00FAEB39FB8A3A8B3B400122753AFF753B95
:100BFC00FF2230600261FE854C50854D51D260431E
:100C0C00E680227892E6FFC3E535948240010FC35B
:100C1C00E53594A040010FC3EF940640027F057E9A
:100C2C00021E3072010EC3E53B940350060E0E30CB
:100C3C0072010EC3E53B940250060E0E3072010E8B
:100C4C00A93BA83A7A04C3E913F9E813F8DAF7C315
:100C5C00E89EF8E99400F94009C3E89402E994008D
:0F0C6C0050047802E4F9E9FBE8FAC3E913FDE864
:100C7B0013FC884C894DC3EF94036037EF20E00DD4
:100C8B00E82CF8E93DF9ECFAEDFB020CABE828F89F
:100C9B00E939F9C3E89402F8E99400F97A02E4FB24
:100CAB00C3EF9403400D8A4E8B4F884889498C4A79
:100CBB008D4B22884E894F8A488B498C4A8D4B220B
:100CCB0030600281CBD26043E680E52D540660276D
:100CDB00A83AA93BE53494085006E820E002A94D58
:100CEB00759100C3E498F594E499F595759104D248
:100CFB006053917F43E68022D265753D00752000DD
:100D0B00020D16D265753D00752040E52D54066029
:100D1B0002C265D2AF206005E53D60012278017A01
:100D2B0002C3E53B940540027802C3E53B940A40BD
:100D3B00027803C3E53B940F40027A0330690478D1
:100D4B001E7A01206007E53D6003D2AF22D2AF00CF
:100D5B0000C2AFC3E53BFB940F40027B0FEB0430AB
:100D6B0073012320620123F93069027982E58BC379
:100D7B009940D0053DEAFBE59B5440B52004DBF7D9
:100D8B00A1B1206502A116C265759100AE3AAF3BC9
:100D9B00C3E49EF594E49FF595759104D26053914D
:100DAB007F43E680A116306502A116D896D2AF22FA
:100DBB0030690B0534206016753400020DD92060A4
:100DCB000D20650A206B07158115810215D222A80B
:100DDB004EA94F75910053917FC3E498F594E49914
:100DEB00F595759104854850854951D26043E6804D
:100DFB002278003064053065027801E53575F0071F
:100E0B00A4F9E5F028F5F0E9A2F013A2F113A2F290
:100E1B0013F535C394785003753578C3E53595369E
:100E2B004008D266C2B1C287C281306002C135852B
:100E3B004A50854B51D26043E68022C2AFC282C278
:100E4B0086C28030720B9001FF7406D5E0FD020E56
:100E5B005C207D02D282307D02D280759F02753C70
:100E6B0002020F9BC2AF207D02C281307D02C2B154
:100E7B003072179001DCC286207D02C280307D0269
:100E8B00C2827406D5E0FD020E9890013F306206D7
:100E9B00E5256002D287207D03759F03307D0375A6
:100EAB009F01753C03020F9BC2AFC282C286C280F8
:100EBB0030720B9001B97406D5E0FD020EC9207D8E
:100ECB0002D280307D02D282207D03759F01307D5E
:100EDB0003759F03753C04020F9BC2AFC287307230
:100EEB0017900196207D02C282307D02C280C2869D
:100EFB007406D5E0FD020F0690012D30620EE5253C
:100F0B00600A207D02D2B1307D02D281759F0275BD
:100F1B003C05020F9BC2AFC282C286C28030720BED
:100F2B0090016B7406D5E0FD020F36D286207D034F
:100F3B00759F03307D03759F01753C06020F9BC2A5
:100F4B00AF207D02C2B1307D02C28130721F900290
:100F5B002A207D02C282307D02C280207D02C280A7
:100F6B00307D02C2827406D5E0FD020F7B900151E9
:100F7B0030620EE525600A207D02D281307D02D2DF
:100F8B00B1207D03759F01307D03759F03753C0177
:100F9B00C266D2AF2290012BC2B1C287C281C2827C
:100FAB00C286C280C26222788076070876070876EE
:100FBB00010876040876FF0876FF087609087602A2
:100FCB00087601087601788C76010876000876B4ED
:100FDB000876FF0876FF0876FF0876030876FF0889
:100FEB0076010876FF0876250876D008767808769D
:100FFB00C80876040876FF08760108760008767A2A
:10100B0008760A087601227887E6FFC272BF0302D0
:10101B00D2727888C27DE630E102D27DC27E7889B9
:10102B00E630E102D27EC3EF94026008758E01D2E6
:10103B0073021044758E00C273227880E614900000
:10104B00809378A1F67881E6149000809378A2F6CD
:10105B00120FA0227886E61490008D9378A3F612D7
:0E106B000FA022789FE6F8700108C3E89411E8
:1010790040027811E82828F5662566256628F5676F
:1010890025662828F56822789CE67536FF75370CA1
:10109900B402067536A075370AB40306753682752B
:1010A900370522227896E6FA7897E6FB307F047AAC
:1010B900007BFFC3EB9AFCC3948250027C82756F5C
:1010C90000056FEC856FF0A4C3E5F0948040F2222F
:1010D900D27F11AD1206C37A007B007C101206B9CB
:1010E900E5592AFA74003BFBDCF37C04C3EB13FBE0
:1010F900EA13FADCF7FEC27F11AD22E5EF20E60321
:101109007520000520903DFFE520146006901FFF23
:101119001460009304600375EF12C2D353D9BF75ED
:1011290081C043FF801206B475EF0243B203E5B3F1
:10113900240420E702F5B3120FA075803875A4C7FF
:1011490075F1FF75D4DF7590FF75A50075F200750F
:10115900D50075A0FF75A60075F30075D60075B0AA
:10116900E475A71B75F4FF75E241120FB212160D53
:1011790078988670C2AF1206CD1206DD1206C31228
:1011890006E41206C31206EB1206C3121730120642
:10119900CD1206CD1206C8C2AFE4F8F6D8FD78C85C
:1011A90079C8308507D9FBD8F7021C00120FB21293
:1011B900160D11121145115F116E119011AC11AD7F
:1011C90078988670120FA075885075891275C82491
:1011D90075910475D84075A82275B80275E69075A1
:1011E9009B80759D0075D10E75BC5875BB0675BA87
:1011F9001F75E8801206B4D2AF120A2043DA01C281
:10120900D8C2711206CD753001D2617B037A0CE523
:101219005870067A0CDB0221A01206C32070022145
:10122900A0C270E559C3940240E3E52F541F855BC2
:101239005AF55BB55AD7DAD7C26153DACF207E03A4
:1012490043DA20307E0343DA10C2D8C271C2757501
:1012590028001206C8307409C3E528940A4002D24E
:10126900751206B978023074027800C3E5599840BE
:10127900F0C2AF1206DD1206DD1206DDD2AF12068C
:10128900CD7546001206B9788CE6C3940150030265
:101299001361E530C394015003021361207435C30F
:1012A900E55994FF5003021361C2AF1206F2D2AF9F
:1012B9001206C8C3E559940150EFC2AF1206DD12F8
:1012C90006BE1206DDD2AF1206C8C3E55994FF4027
:1012D900E90217B57F05D27F11AD1206C8C2AFC2A8
:1012E9007F11ADAE59C3E559947FD2AF4074120650
:1012F900B4C2AF1206F2D2AFDFDC11D9C3EE940546
:101309007897F61206CD12164F1217387F0AD27F38
:1013190011AD1206C8C2AFC27F11ADAE59C3E559AE
:10132900947FD2AF50E61206B4C2AF1206DD1206A0
:10133900BE1206DDD2AFDFD611D9EE24057896F6B6
:101349001206CD12164F1217671206C811ADC3E562
:101359005994FF40F40217B5C3E5599546400385F2
:1013690059461206C878017988E7B403027805C39B
:10137900E559984002418DC2AF1206F21206F212E7
:1013890006F2D2AF1206CD753000E4F531F532051B
:1013990031E531F470390532789AE678191460121A
:1013A900783214600D787D14600878FA146003753A
:1013B9003200C3E53298401715327531B4789986F1
:1013C90070C2AF1206F2D2AF789886701206C812B0
:1013D90006BEE529700530740221A0780120740247
:1013E9007806C3E5599840A71206C8E52970022175
:1013F900A0C2AF120FA0E4F522F523F524F525D2FA
:10140900AF78858662F53EF53FF540F541F542F541
:101419006DF547F52CF52DF535120B92756D08759F
:10142900BB1E1206B4120ABBE5E820ECFBA8BDA955
:10143900BEE97001F8886E120ABF756D0875BB1E8A
:101449007887E6FE760211127887EEF6C2AF755EEE
:10145900FF120B7485225E85225F852260D2AF75EB
:0E1469002201752401752501855D64756501FC
:10147700D268D269753400120F20120F4A120B92EC
:10148700120B99120C0F02149B120FA01112756DFB
:101497000075BB06120D0E120DBB120DDA1207DC1A
:1014A700120DFC120E46120B99120BFE120C0F12A4
:1014B7000CCB120D03120DBB120DDA12087F1209A5
:1014C700E4120DFC120E6F120B99120BFE120C0F89
:1014D700120CCB120D0E120DBB120DDA1208BF1231
:1014E7000DFC120EB3120B99120BFE120C0F120CFD
:1014F700CB120D03120DBB120DDA12091C120DFCD3
:10150700120EE5120B99120BFE120C0F120CCB12D6
:101517000D0E120DBB120DDA120981120DFC120FFE
:1015270020120B99120BFE120C0F120CCB120D038B
:10153700120ABB120DBB120DDA120ABF120DFC12F2
:101547000F4A120B99120BFE120C0F120CCB3069BB
:101557002F206B2C85615E85615F855D64756501F4
:1015670079327A0AC3E534994009C269D26A8A3363
:10157700021587C3E5599401400302149B0215D253
:10158700306A1B206B18E533147004C26A8190F52A
:1015970033C3E5599401400302149B0215D2C3E5F6
:1015A7005C9401400985615F855D64756501C3E5EC
:1015B7005C94FA5016307404E529600FC3E53B7854
:1015C700F0306B027860985002819BC2AF120FA077
:1015D7007887E6FE760211127887EEF6E4F522F5B3
:1015E70023F524F525F562C268D2AF1206B4120FAF
:1015F700A0307406E529700221A0788DE6C3940116
:101607004002416A6193901A0D7820121691E520E5
:10161700B4A50CA3121691E520B45A0302162F1293
:101627000FB212164F02164E901A0378807B0A12D9
:101637001691A308DBF9901A0F788C7B1512169177
:10164700A308DBF9901A2422C2AF1216D01216AAE9
:10165700901A00740D121696A37402121696A374AC
:1016670013121696901A0378807B0A121695A30810
:10167700DBF9901A0F788C7B15121695A308DBF906
:101687001216E31216C1901A2422E493F622E643B7
:101697008F01538FFD75EF0275B7A575B7F1F0533D
:1016A7008FFE22438F02438F0175EF0275B7A57531
:1016B700B7F1901A0DF0538FFC22901A0D74A5D133
:1016C70096901A0E745AD196227A3079D078209053
:1016D7001A40D191E520F709A3DAF7227A3079D0B9
:1016E700901A40E7D19609A3DAF922AB71A872BB29
:1016F70001027980BB02027981BB03027982BB04B4
:10170700027994BB05027983BB06027986BB07027F
:101717007992BB08027987BB0902799CBB0A0279D7
:1017270088BB0B027989E8F7227C051206CDDCFB22
:1017370022C2AF1206DD1206E41206EB1206F212FF
:1017470006BE1206DD1206E41206EB1206F21206B8
:10175700BE1206DD1206E41206EB1206F2D2AF2223
:10176700C2AF1206F21206EB1206E41206DD1206EB
:10177700BE1206F21206EB1206E41206DD1206BED0
:101787001206F21206EB1206E41206DDD2AF22AE03
:1017970071AF72C2AF1206DD1206DD1206DD120648
:1017A700BEDEF21206F21206BEDFF8D2AF22F13821
:1017B700F130F130757101757201757300F1967C26
:1017C70005AD591206CDC3ED955970F5C3E559948A
:1017D70001400AC3E55994FF40330217F1D1F2D112
:1017E7004FF138C2AF75EF12F130DCD50573C3E5A1
:1017F700739403500280C61217300572E571149076
:10180700009A93F808C3E57298500280AD1217301A
:101817001217300571C3E571940C50028099120FAD
:0C182700B212164FC2AF75EF121217304C
:101A00000D021307070104FFFF09020101A55A0196
:101A100000B4FFFFFF03FF01FF25D078C804FF01DA
:051A200000FF0A01FFB8
:101A4000235475726E696779343041232020202039
:101A500023424C48454C4923463331302320202033
:101A60002020202020202020202020202020202076
:101C0000C2AFC2D353D9BF7581C043B20343FF8073
:101C1000752438752503B1BF75EF0275E24043F1B5
:101C20002053A4DFD285780379E67C1075220075F5
:101C30002300901DCC7B0675249875250130850204
:101C4000813D208508D8FBD9F9DCF781AD308508C6
:101C5000D8FBD9F9DCF781ADB17FE493A3C39A60D7
:101C6000028126DBDDB171600281267B08E493FAF4
:101C7000A3B152DBF87A30B152752200752300B15E
:101C800071EAFCEBFDC3ED94FE400EB1718A278B27
:101C900028ED30E0048A828B83B1717AC270D8C398
:101CA000ED94FE601050CEBD0022EC600675200061
:101CB0000200008100A827A9280809D804D90281B8
:101CC000C9B175EA89AAF281BB0D8199C3ED94036C
:101CD0005049EDA2E092007AC5C3E5829400E58305
:101CE000941C5093200010438F02438F0175B7A5B9
:101CF00075B7F1F030001FA827A9280809438F0104
:101D0000538FFDD804D902A11689AAE275B7A5752B
:101D1000B7F1F0A3A103538FFC81757AC1BD030C09
:101D2000E493A3FAB136DCF8B12E81758177AA224B
:101D3000AB23B152EBFAEA6222752608C3E52313FE
:101D4000F523E52213F52250066323A0632201D573
:101D500026EAB1BFB1BF75260AEAF4200102D28596
:101D6000300102C285B1BFC3134002C201D526EBC8
:101D700022B175EAFB208502A175308502A17A7532
:101D80002608AE24AF25C3EF13FFEE13FEB1C3B197
:101D9000BFC3EA133085024480FA30E703632201AF
:101DA000C3E52313F523E52213F52250066323A090
:101DB000632201D526D9E52265236523F52222AECB
:101DC00024AF250E0FDEFEDFFCD20122424C486517
:0A1DD0006C6934373132F31006015C
:00000001FF
